:0200000480007A
:10000000130E100013000000130000001300000086
:1000100013000000537110001300000013000000D3
:1000200013000000130000006F00800113000000A7
:100030001300000013000000130000001300000074
:10004000130E20009700000083A0802E5371100033
:100050001300000013000000130000001300000054
:100060006F000002130000001300000013000000E6
:100070001300000013000000130000001300000034
:10008000130E3000130000001300000013000000E6
:10009000130000006F008000537110006F004002D9
:1000A0001300000013000000130000001300000004
:1000B00013000000130000001300000013000000F4
:1000C000130E400013000000130000001300000096
:1000D00013000000970000009380802507A1000016
:1000E00013000000130000001300000013000000C4
:1000F0006F00000113000000130000001300000057
:10010000130E500013000000130000001300000045
:100110001300000097000000938080211701000069
:100120001301412187A0000007210100D3F1200025
:100130001300000013000000130000001300000073
:100140006F00000413000000130000001300000003
:100150001300000013000000130000001300000053
:100160001300000013000000130000001300000043
:100170001300000013000000130000001300000033
:10018000130E6000130000001300000013000000B5
:1001900013000000970000009380001A27A0300091
:1001A0001300000013000000130000001300000003
:1001B0006F00000113000000130000001300000096
:1001C000130E7000970000009380001717010000C5
:1001D0001301C116970100009381811617020000D8
:1001E0001302421607A2000053724200D3F24000ED
:1001F0002720410027A051002720120013000000F3
:100200001300000013000000130000006F00400303
:100210001300000013000000130000001300000092
:100220001300000013000000130000001300000082
:100230001300000013000000130000001300000072
:10024000130E8000D3F011C0130000001300000053
:1002500013000000130000006F0080021300000074
:100260001300000013000000130000001300000042
:100270001300000013000000130000001300000032
:10028000130E9000D30031A0538121A0D38131A05F
:100290001300000013000000130000001300000012
:1002A0006F000002130000001300000013000000A4
:1002B00013000000130000001300000013000000F2
:1002C000130EA00093000001D3F010D01301200101
:1002D00093010020537111D0D3F111D01702000007
:1002E0000322420AD37212D0130000001300000050
:1002F00013000000130000006F000001370110F030
:10030000130141F22320C101370110F0130101F262
:100310002320010013000000130000001300000060
:100320001300000013000000130000000000C03F95
:100330000000A040490000003A0000003800000022
:100340004B00000013000000130000001300000029
:100350001300000013000000130000001300000051
:100360001300000013000000130000001300000041
:100370001300000013000000130000001300000031
:10038000D401000000000000000000000000000098
:10039000000000000000000000000000000000005D
:1003A000000000000000000000000000000000004D
:0803B000000000000000000045
:00000001FF
